:100000000C9494010C94BC010C94BC010C94BC01A4
:100010000C94BC010C94BC010C94BC010C94BC016C
:100020000C94BC010C94BC010C94B11A0C947D1975
:100030000C94BC010C94BC010C94BC010C94BC014C
:100040000C94BC010C94370A0C94BC010C94BC01B8
:100050000C94BC010C94BC010C94BC010C94FD12DA
:100060000C94BC010C94BC010C94BC010C94BC011C
:100070000C94BC010C94BC010C94BC010C94BC010C
:100080000C94BC010C94BC010C94BC010C94BC01FC
:100090000C94F90D0C94BC010C94BC010C94BC01A3
:1000A0000C94BC010C94BC010C94BC017D09990911
:1000B000BD0899092E0999099B084A0899099909C7
:1000C00099099909990961079909300899098208DC
:1000D000541459145E1468147214BC14BC14BC1467
:1000E0007C14861490149A14A714BC14AF14DD1455
:1000F000E014CF14D314D914011501150115E4141B
:10010000E814EC14F214F6140115FC1407060504A7
:100110000100080A0B0C0D090000000200090F0085
:1001200000030401000C00000000000000000000BB
:100130000000000000000408020110408040102070
:10014000408040800802040180402010020110809D
:1001500010204040040404040403040502020202C7
:100160000403020202020606060606060404020250
:100170000204000000002300260029002C002F00AC
:1001800000000000250028002B002E003100000098
:100190000000240027002A002D003000080B000278
:1001A000020201000904000001020200000524000F
:1001B00010010524010101042402060524060001A2
:1001C0000705810310004009040100020A00000035
:1001D000070502024000000705830240000000C13D
:1001E0008081C11201000202000040EB03042400E0
:1001F00001010200011201000200000040EB0304B3
:100200002400010102000152424C00426C656E6400
:10021000204D6963726F00040309040000000000B0
:100220000000002A2B280000000000000000000051
:1002300000000000000000000000002C9EB4A0A1FF
:10024000A2A434A6A7A5AE362D3738271E1F20211D
:100250002223242526B333B62EB7B89F84858687FC
:1002600088898A8B8C8D8E8F909192939495969796
:1002700098999A9B9C9D2F3130A3AD3504050607B4
:1002800008090A0B0C0D0E0F101112131415161776
:1002900018191A1B1C1DAFB1B0B5000904020001EA
:1002A0000300000009210101000122650007058407
:1002B0000340000105010902A1010901A100850116
:1002C000050919012903150025019503750181020E
:1002D000950175058103050109300931093815813A
:1002E000257F750895038106C0C005010906A10197
:1002F0008502050719E029E7150025017501950814
:10030000810295017508810395067508150025651C
:100310000507190029658100C000C606170DD71210
:10032000DB125D16C016A51C11241FBECFEFDAE04C
:10033000DEBFCDBF11E0A0E0B1E0E8E1FDE302C027
:1003400005900D92A43FB107D9F724E0A4EFB1E0E6
:1003500001C01D92A83BB207E1F713E0C8E2D3E069
:1003600004C02297FE010E94111DCA31D107C9F7AE
:100370000E94E6120C948A1E0C9400001F93CF93E7
:10038000DF93162F843008F06CC0982F990F990FC7
:10039000990F985F9F3108F09EE1D82FDD0FDD0F98
:1003A000DD0F8D2FC0E041E08917C8F4E82FF0E0A1
:1003B000DF01A053BD4F2C91223070F4C42BEE0FFF
:1003C000FF1FE057FD4F21E030E0542F512311F47F
:1003D00020E030E031832083440F8F5FE5CFC0FF02
:1003E00005C0612F61708D2F0E943B15C1FF06C0B3
:1003F000612F627081E08D0F0E943B15C2FF06C025
:10040000612F647082E08D0F0E943B15C3FF06C010
:10041000612F687083E08D0F0E943B15C4FF06C0FA
:10042000612F607184E08D0F0E943B15C5FF06C0EF
:10043000612F607285E08D0F0E943B15C6FF06C0DC
:10044000612F607486E08D0F0E943B15C7FF09C0C5
:10045000612F607887E08D0FDF91CF911F910C9411
:100460003B15DF91CF911F9108950F931F93CF9369
:10047000DF93EB018E3178F5082F10E0F801E0539F
:10048000FD4F9081933089F0943029F5F801ED5FAC
:10049000FD4F208130E0C901880F991F820F931F03
:1004A0008F5D9D4F0E94D20B0FC0833051F09BEFA8
:1004B000980F923030F097EF980F933010F08D3006
:1004C00019F4BE010E942E14F801EE0FFF1FE05731
:1004D000FD4FD183C083DF91CF911F910F9108957C
:1004E000CF93C82F8C3058F54091F6025091F70207
:1004F00021E030E0082E02C0220F331F0A94E2F7F9
:10050000672B49F420953095242335233093F70247
:100510002093F60214C0242B352B3093F70220933E
:10052000F6028091F40181110AC08C2F0E94FD1304
:10053000AC016C2F8EED93E0CF910C94A110CF9174
:100540000895DB019A019091F5019C30D0F540911E
:10055000F601682F70E0442369F0E42FF0E0EA50E0
:10056000FE4F8081FB01ED5FFD4F80834150409342
:10057000F60107C0FB01ED5FFD4F90839F5F9093F5
:10058000F501FB01ED5FFD4F1A161B067CF41216F8
:10059000130664F4408150E0CA01880F991F840F4C
:1005A000951FAD018F5D9D4F0C940F0B208130E0A6
:1005B000C901880F991F820F931F8F5D9D4F0C9467
:1005C0008D0B68E171E08EED93E00C943011CF93C8
:1005D000DF93C82FD0E0CD5FDD4F288130E0C90127
:1005E000880F991F820F931F8F5D9D4F0E94930B61
:1005F00088819091F501891306C0882379F0815094
:100600008093F5010BC0992349F0E091F601EF5F6B
:10061000E093F601F0E0EA50FE4F80838FEF88838D
:10062000DF91CF9108951F93CF93DF93162FC82F9B
:10063000D0E0FE01E453FD4F90811923C251DD4FFC
:10064000411103C09881911741F0412F50E0682F6C
:100650008EED93E00E94BA101883DF91CF911F9125
:100660000895EF92FF920F931F93CF93DF93E82E9D
:1006700083E08E1508F475C02E2D30E0F901EE50A0
:10068000FD4F6083672B09F46CC0F901E453FD4F03
:10069000F0800E2D000F000F000FF0FE52C0802FD3
:1006A0000E947115892B09F44CC011E0C02FD0E0D5
:1006B000F1FE07C081E0800F0E947115892B09F0BF
:1006C00042C0F2FE06C082E0800F0E947115892BA5
:1006D000E1F5F3FE06C083E0800F0E947115892BBF
:1006E000B1F5F4FE06C084E0800F0E947115892BDD
:1006F00081F5F5FE06C085E0800F0E947115892BFB
:1007000051F5C831D10541F0F6FE06C086E0800FF4
:100710000E947115892B09F5679744F4F7FE06C00E
:1007200087E0800F0E947115892BC9F441E0612F89
:100730008E2DDF91CF911F910F91FF90EF900C9430
:10074000130310E0B3CF1260BCCF1460C2CF1860A7
:10075000C8CF1061CECF1062D4CF1064DDCF106847
:10076000E5CFDF91CF911F910F91FF90EF9008950A
:10077000CF93DF938091F202882309F448C0D0918F
:10078000CC02D0FF1DC180E00E947115892B09F4B5
:1007900017C1C1E0D1FF06C081E00E947115892B0D
:1007A00009F010C1D2FF06C082E00E947115892BAA
:1007B00009F00AC1D3FF06C083E00E947115892B9E
:1007C00009F004C1D4FF06C084E00E947115892B92
:1007D00009F0FEC0D5FF06C085E00E947115892B87
:1007E00009F0F8C0D6FF06C086E00E947115892B7B
:1007F00009F0F2C0D7FF06C087E00E947115892B6F
:1008000009F0ECC040E06C2F80E00E94130380915F
:10081000F302882309F448C0D091CD02D0FFE0C094
:1008200088E00E947115892B09F4DAC0C1E0D1FF7C
:1008300006C089E00E947115892B09F0D3C0D2FF50
:1008400006C08AE00E947115892B09F0CDC0D3FF44
:1008500006C08BE00E947115892B09F0C7C0D4FF38
:1008600006C08CE00E947115892B09F0C1C0D5FF2C
:1008700006C08DE00E947115892B09F0BBC0D6FF20
:1008800006C08EE00E947115892B09F0B5C0D7FF14
:1008900006C08FE00E947115892B09F0AFC040E0BF
:1008A0006C2F81E00E9413038091F402882309F4E5
:1008B00048C0D091CE02D0FFA3C080E10E94711544
:1008C000892B09F49DC0C1E0D1FF06C081E10E94DF
:1008D0007115892B09F096C0D2FF06C082E10E94F3
:1008E0007115892B09F090C0D3FF06C083E10E94E7
:1008F0007115892B09F08AC0D4FF06C084E10E94DB
:100900007115892B09F084C0D5FF06C085E10E94CE
:100910007115892B09F07EC0D6FF06C086E10E94C2
:100920007115892B09F078C0D7FF06C087E10E94B6
:100930007115892B09F072C040E06C2F82E00E9493
:1009400013038091F502882309F476C0D091CF0279
:10095000D0FF66C088E10E947115892B09F460C040
:10096000C1E0D1FF06C089E10E947115892B09F011
:1009700059C0D2FF06C08AE10E947115892B09F087
:1009800053C0D3FF06C08BE10E947115892B09F07B
:100990004DC0D4FF06C08CE10E947115892B09F06F
:1009A00047C0D5FF06C08DE10E947115892B09F063
:1009B00041C040E06C2F83E0DF91CF910C94130392
:1009C000C0E0E8CEC260EECEC460F4CEC860FACE1D
:1009D000C06100CFC06206CFC0640CCFC06812CF28
:1009E000C0E025CFC2602BCFC46031CFC86037CF05
:1009F000C0613DCFC06243CFC06449CFC0684FCF14
:100A0000C0E062CFC26068CFC4606ECFC86074CFF0
:100A1000C0617ACFC06280CFC06486CFC0688CCFFF
:100A2000C0E09FCFC260A5CFC460ABCFC860B1CFDC
:100A3000C061B7CFC062BDCFDF91CF910895109252
:100A400047028FEF80930A010895CF92DF92EF92D1
:100A5000FF920F931F93CF93DF93182FEB01E82E94
:100A6000F12CC70180539D4F6C01FC0180818F37B1
:100A700009F4EEC0863051F480914702882331F0AA
:100A80006630710509F4E0C00E941F051E31A8F40C
:100A9000C430D10591F0F701ED5FFD4F20812C307E
:100AA00060F430E0C901880F991F820F931F8F5D9A
:100AB0009D4F0E94370C8111B4C00EEE010F0C3017
:100AC00058F461E070E0C230D10511F060E070E0F0
:100AD000802F0E94700202C01E31D0F4E12FE695F3
:100AE000E695E695812F8770F0E0E453FD4F21E015
:100AF00030E0082E01C0220F0A94EAF7209721F473
:100B00008081822B808304C02095808128232083CC
:100B1000F701EE0FFF1FE057FD4F11821082C23028
:100B2000D10579F02CF42097C9F0219729F16BC0F9
:100B3000C430D10509F445C064F1269709F45BC0BF
:100B400062C00C3008F084C060E0812F0E94021562
:100B500060E0812F0E943B1582E052C01E3108F0F8
:100B600077C060E0812F0E94021560E0812F0E9413
:100B70003B15F60110826CC01E3108F069C060E0C0
:100B8000812F0E943B1561E0812F0E94021581E0B8
:100B900037C0133059F08BEF810F823038F087EF78
:100BA000810F833018F01D3009F052C061E0812FB1
:100BB0000E94021560E070E0812F0E942E1483E0F5
:100BC0001FC01E3108F044C084E0F6018083F701A5
:100BD000ED5FFD4F80818F3F41F190E09C01220F3E
:100BE000331F280F391FC9018F5D9D4F0E94370C9D
:100BF00081112EC01AC08EEF810F823048F586E039
:100C0000F601808325C06CE271E08EED93E0DF9108
:100C1000CF911F910F91FF90EF90DF90CF900C94A8
:100C20003011812F0E94E70248CF4FEF5FEF6FEF47
:100C30007FEF812FDF91CF911F910F91FF90EF9068
:100C4000DF90CF900C94A1021E3108F424CF35CF51
:100C5000DF91CF911F910F91FF90EF90DF90CF9098
:100C60000895CF93C0E08EEF8C0F823028F466E0B9
:100C700070E08C2F0E942505CF5FCE31A1F781E077
:100C8000809347028EE193E0CF910C94DD0C0F939B
:100C90001F93CF93DF9381E08093F401809147020B
:100CA00081110E941F05E2EFF2E0CCECD2E0AEEE43
:100CB000B2E0119219921D9282E0E63FF807C9F75F
:100CC000C3E0D2E010E00FEF8EEE810F8C3018F40D
:100CD00062E070E002C061E070E0812F0E942505B3
:100CE00009931F5F1E3181F71092F7021092F602EE
:100CF0001092F6011092F5011092F401DF91CF915C
:100D00001F910F91089524E042E06DE371E08EEDB4
:100D100093E00E94C80F45E352E060EE8EED93E051
:100D20000E943E114EEB51E060E98EED93E00E948F
:100D30003E1140E752E060EC8EED93E00E943E11E0
:100D400041E353E060ED8EED93E00E943E1145E2F9
:100D500055E064EF8EED93E00E943E114DE457E0C4
:100D600060EF8EED93E00E94691147E456E06FEF6B
:100D70008EED93E00E94611140E051EE60E070E082
:100D80008EED93E00E94C1120C944706CF93DF933F
:100D9000C1E2D2E0CE010E94F30A239682E0C5347C
:100DA000D807C1F7DF91CF910895682F8EE193E0C6
:100DB0000C949E0C8EE193E00E944E0C0895DF92FD
:100DC000EF92FF920F931F93CF93DF93F82EEB01D7
:100DD000D42E6F3F8FEF7807A9F06F2D8EE193E04F
:100DE0000E94F70C8C2F0E94D5068EE193E00E94A2
:100DF000140D8091450290914602009729F00E94BF
:100E00009E1302C0C0E0D0E04D2D6F2D8EE193E027
:100E10000E94F40C0D2D10E08EE193E00E94460C30
:100E2000081719071CF461E571E009C08EE193E031
:100E30000E94460C8017910734F46EE671E08EED47
:100E400093E00E943011F0924802C09349028AE474
:100E5000E82E82E0F82EC0E0D0E0C017D10784F081
:100E600042E04D0D28E432E067E78EED93E0DF913C
:100E7000CF911F910F91FF90EF90DF900C94E810AD
:100E80008EE193E00E94460C892B51F30E94DA0612
:100E9000F70181937F012196E0CFEF92FF920F93AC
:100EA0001F93CF93DF93162FEA0190E0FC01E956E0
:100EB000F109E231F10508F03CC2EA5AFF4F0C9407
:100EC0000F1D8981982F987185FF03C06AE871E032
:100ED00056C08881983071F148F491112AC2682F68
:100EE0008EE193E00E94F70C02E007C0903109F414
:100EF00040C0983109F471C01CC2011768F4FE01AA
:100F0000E00FF11D9181808120E8929F80191124CA
:100F10000E94D5060E5FF1CF8EE193E00E94140D82
:100F200086E490E0DF91CF911F910F91FF90EF90B9
:100F30000C949E134A816B81163069F430E8639FEC
:100F4000B0011124640F711D9D814C8150E8959F63
:100F50004019112406C090E8699F401911246FEFD1
:100F60007FEFDF91CF911F910F91FF90EF900C9445
:100F7000DF06E0910A01E73064F06AEA71E08EED85
:100F800093E0DF91CF911F910F91FF90EF900C9420
:100F900030119A812B81F0E8663061F42F9F900127
:100FA0001124290F311D4D819C8150E8459F9019D6
:100FB000112405C02F9F901911242FEF3FEFEF5FF1
:100FC000E0930A0144E0E402F0011124E859FD4FE6
:100FD0008083328321839383ACC150910A0115161B
:100FE00034F440E0252F332727FD30950EC08FEFD6
:100FF00080930A019EC1EE0FFF1FEE0FFF1FE859FD
:10100000FD4F9081981719F14F5FE42FF0E02E17F4
:101010003F078CF740E01BC04830C0F4DF01AA0F47
:10102000BB1FAA0FBB1FA459BD4F8C91EE0FFF1F12
:10103000EE0FFF1FE859FD4F808311968D919C9113
:1010400012979283818313968C9183834F5FE42F51
:10105000F0E02E173F0704F7515050930A0169C181
:101060002881898150E8859FC0011124820F911D3C
:10107000009721F0909346028093450280914702A9
:10108000811157C1DF91CF911F910F91FF90EF9088
:101090000C943106653008F44CC118810981FA803E
:1010A000EB80CC811E3108F044C1E12FF0E0ED5F10
:1010B000FD4FE081EC3060F4F0E0CF01880F991F24
:1010C0008E0F9F1F8F5D9D4F0E94370C81112DC188
:1010D00080E8C89FA00111244E0D511D90E8F99E93
:1010E000B0011124600F711D812F0E94A10264E0E4
:1010F00070E0812FDF91CF911F910F91FF90EF90C2
:101100000C942505623008F414C128818981E0E837
:101110008E9FC0011124820F911D90930C0180932A
:101120000B010A9708F005C18AE090E090930C014A
:1011300080930B01FEC0623008F4FBC0698170E04F
:10114000123091F08A81F0E88F9FC0011124682B42
:10115000792B133049F08B8190E090E4899F902D9A
:1011600088271124682B792B8881DF91CF911F91DB
:101170000F91FF90EF900C94350260EF8EED93E0AD
:101180000E9434116CE68EED93E00E943411C0E0B1
:1011900060E08EED93E00E94341161E08EED93E00B
:1011A0000E94341161E08EED93E00E94341161E001
:1011B0008EED93E00E9434118EEE8C0F8C3058F43B
:1011C00062E08EED93E00E9434116AE08EED93E0D0
:1011D0000E9434110DC0C33059F463E08EED93E0EA
:1011E0000E94341168E08EED93E00E9434110AC031
:1011F0008BEF8C0F823088F387EF8C0F833068F38E
:10120000CD3059F364E08EED93E00E9434116EE02E
:101210008EED93E00E9434118EEF8C0F823050F4EB
:1012200066E08EED93E00E94341161E08EED93E074
:101230000E9434116FE78EED93E00E943411CF5F6E
:10124000CE3109F0A5CF67EF8EED93E0DF91CF911E
:101250001F910F91FF90EF900C943411662309F4C5
:1012600068C0C88160EF8EED93E00E9434116EE695
:101270008EED93E00E9434116C2F8EED93E00E946E
:101280003411CE3100F7D0E0FE01E053FD4F608114
:101290008EED93E00E943411CC0FDD1F8E010057BC
:1012A0001D4FF80160816F778EED93E00E9434113D
:1012B000F80160817181CB018078892B49F0660F3C
:1012C000672F661F770B6F778EED93E00E943411C6
:1012D000C057DD4F68817981CB018827907C892BAD
:1012E00009F4B1CF770F660B770F762F661F6F77F4
:1012F0008EED93E00E943411A6CF60EF8EED93E067
:101300000E9434116AE68EED93E00E943411CEEE15
:10131000CC3010F06FE701C06C2F8EED93E00E948F
:101320003411CF5FCC30A1F78ECF812F0E94E7021E
:10133000CFCEDF91CF911F910F91FF90EF90089545
:101340008F929F92AF92BF92CF92DF92EF92FF92D5
:101350000F931F93CF93DF930E94B8038EED93E01A
:101360000E942810892B29F08EED93E00E949411A1
:10137000F5CF0E94471360938C0270938D02809387
:101380008E0290938F02C0908802D0908902E090E4
:101390008A02F0908B0240910B0150910C014A019E
:1013A000A12CB12C8B019C010C191D092E093F09A0
:1013B00080169106A206B30608F04CC0D501C40100
:1013C0008C0D9D1DAE1DBF1D8093880290938902D8
:1013D000A0938A02B0938B02C0EDD2E01EEE1C30C7
:1013E000C0F488818230A9F42091F6023091F7028E
:1013F000012E02C0359527950A94E2F720FF09C017
:10140000812F0E94FD13AC01612F8EED93E00E94AD
:10141000A1101F5F21961C3011F780910A0187FDF2
:1014200019C0C0E0EC2FF0E080910A01992787FDF8
:1014300090958E179F0774F0EE0FFF1FEE0FFF1FA2
:10144000E859FD4F61817281438180810E94DF06EE
:10145000CF5FE8CFDF91CF911F910F91FF90EF9079
:10146000DF90CF90BF90AF909F908F9008951F9284
:101470000F920FB60F9211242F933F934F935F93C8
:101480006F937F938F939F93AF93BF93EF93FF934C
:101490008091F90287FF05C01092850010928400A8
:1014A0001AC02091F902332727FD30958091F80268
:1014B00090E0281739077CF48091F902992787FD7D
:1014C0009095FC01EE0FFF1FE80FF91FE650FD4F4E
:1014D000808186FD15C08091F9028F5F8093F902AB
:1014E0002091F902332727FD30958091F80290E092
:1014F00028173907BCF48091F9028C305CF112C0D6
:101500008091F902992787FD9095FC01EE0FFF1F4E
:10151000E80FF91FE650FD4F808160E08F730E9455
:101520003B15D9CF8091840090918500049680323C
:101530009E4418F480E29EE405C08091840090915E
:101540008500049690938900809388008FEF8093A4
:10155000F90238C020918400309185008091F90211
:10156000992787FD9095FC01EE0FFF1FE80FF91FEB
:10157000E650FD4F81819281820F931F90938900E5
:10158000809388008091F902992787FD9095FC014E
:10159000EE0FFF1FE80FF91FE650FD4F808186FF19
:1015A00011C08091F902992787FD9095FC01EE0FFB
:1015B000FF1FE80FF91FE650FD4F808161E08F7338
:1015C0000E943B15FF91EF91BF91AF919F918F9139
:1015D0007F916F915F914F913F912F910F900FBE2F
:1015E0000F901F9018952091F8022C30A0F431E054
:1015F000320F3093F802FC012083822F90E0FC012F
:10160000EE0FFF1FE80FF91FE650FD4F8CED95E040
:101610009283818308952FEFFC0120830895DF9248
:10162000EF92FF920F931F93CF93DF93EC01D62E8F
:101630007A01890188818C3008F066C061E08D2DC7
:101640000E9402158881A82FB0E0FD01EE0FFF1F58
:10165000EA0FFB1FE650FD4F2D2D2F739081907CDC
:10166000922B908360E272E06E197F0977FF02C0CF
:101670006D5F7F4F7595679575956795698340E6B2
:1016800059E0401B510B57FF02C04D5F5F4F55950E
:101690004795559547954A836CE00E94C21C9CE093
:1016A000899FB001112420E030E0A901460F571FA7
:1016B000FA01EE0FFF1FE40FF51FE650FD4F90817A
:1016C00096FD16C02F5F3F4F2C30310571F7811109
:1016D0000FC01092800082E08093810010928500FC
:1016E00010928400B19A80916F00826080936F00A5
:1016F000888190E0FC01EE0FFF1FE80FF91FE65014
:10170000FD4F8081806480838881DF91CF911F911C
:101710000F91FF90EF90DF90089520E639E040E2CE
:1017200052E00C940F0BFC01808190E0FC01EE0F65
:10173000FF1FE80FF91FE650FD4F80818F7B8083EC
:101740000895FC0180818C3060F5918128E830E0BB
:10175000291B310997FD3395220F331F220F331FA9
:10176000621773077CF0928128E532E0291B31096A
:1017700097FD3395220F331F220F331F6217730714
:101780000CF49B014FB7F89490E022503109FC0112
:10179000EE0FFF1FE80FF91FE650FD4F3283218344
:1017A0004FBF08954F925F926F927F92AF92BF9218
:1017B000CF92DF92EF92FF920F931F93CF93DF931D
:1017C000EC01603282E078070CF040C077FD06C083
:1017D000653B71052CF064EB70E002C060E070E0E6
:1017E000898128E830E0281B310987FD3395220FD5
:1017F000331F220F331F5901CC24B7FCC094DC2CBB
:10180000882777FD8095982F2A8148E552E0421B72
:10181000510927FD5395440F551F440F551F2A01A9
:10182000662457FC6094762C7F926F925F924F9261
:1018300014EBE12EF12C00E010E020E030E0A901F3
:101840000E94271B0F900F900F900F90CE01DF91F9
:10185000CF911F910F91FF90EF90DF90CF90BF90AD
:10186000AF907F906F905F904F900C94A10BFC0114
:10187000808190E0FC01EE0FFF1FE80FF91FE6509A
:10188000FD4F808186FB882780F9089580914E0363
:1018900090E020914F03821B9109089520914F03FE
:1018A00080914E03281750F4E22FF0E0E05BFC4FEC
:1018B000808190E02F5F20934F0308958FEF9FEF7B
:1018C0000895E0914F0380914E03E81730F4F0E063
:1018D000E05BFC4F808190E008958FEF9FEF0895CB
:1018E0000895CF92DF92EF92FF920F931F93CF93C1
:1018F000DF937C01CB018A0120912A03222389F006
:10190000EB016B01C40ED51ECC15DD0569F06991A4
:10191000D701ED91FC910190F081E02DC70109956F
:10192000F3CF642F0E94D00DC801DF91CF911F919A
:101930000F91FF90EF90DF90CF900895CF93DF93BA
:101940001F92CDB7DEB7698320912A032223D1F0FD
:1019500020912B03203240F021E030E0FC01338362
:10196000228380E090E015C080912C03E82FF0E006
:10197000E35DFC4F998190838F5F80932C0380936C
:101980002B0305C061E0CE0101960E94D00D81E0DD
:1019900090E00F90DF91CF910895FC0113821282A5
:1019A00048EE53E060E070E04483558366837783BC
:1019B0008FEB91E091838083089510924F031092F2
:1019C0004E0310922C0310922B030C941B0D862FA8
:1019D000413208F040E260E573E00E94390D109258
:1019E0004F0380934E03089521E00C94E70C81E0AF
:1019F00080932A0360934D0310922C0310922B03C3
:101A000008950F93062F21E040912B036DE273E0C0
:101A100080914D030E947D0D10922C0310922B0398
:101A200010922A030F91089561E00C94010D8EE14C
:101A300093E00C94CD0C1092DD0381E08093DB03E6
:101A40001092DA0361E082E00E943B1561E083E0DE
:101A50000E943B15E9EBF0E080818E7F80838081DE
:101A60008D7F808380E28093B80085E48093BC0002
:101A70000895413208F03FC09091DD039111FCCFF1
:101A800091E09093DD032093DB032FEF209370030D
:101A90001092B503240F2093B4039093DC0390912C
:101AA000DC03880F892B8093DC038091DA0381307B
:101AB00041F41092DA038091DC038093BB0085EC43
:101AC00001C085EE8093BC008091DD038130E1F39D
:101AD0008091B503841710F44091B50326EB33E0F1
:101AE000FB01D9018A2F821B841718F48D918193F1
:101AF000F9CF842F089580E008950F93413208F0C4
:101B000046C09091DD039111FCCF92E09093DD03EC
:101B10000093DB039FEF909370031092B503409303
:101B2000B403FB0166EB73E0DB019A2F961B94175D
:101B300018F491919D93F9CF1092DC039091DC03FE
:101B4000880F892B8093DC038091DA03813041F484
:101B50001092DA038091DC038093BB0085EC01C016
:101B600085EE8093BC00222321F08091DD0382303A
:101B7000E1F3809170038F3F61F0809170038032B8
:101B800051F080917003803341F483E007C081E01D
:101B900005C080E003C082E001C084E00F91089599
:101BA000613298F42091DD03243089F4609392032C
:101BB000FC0184E993E0DC012A2F281B261718F486
:101BC00021912D93F9CF80E0089581E0089582E07E
:101BD000089585ED8093BC008091BC0084FDFCCF0E
:101BE0001092DD03089585EC8093BC001092DD0314
:101BF00008951F920F920FB60F9211242F933F93C7
:101C00004F935F936F937F938F939F93AF93BF9304
:101C1000EF93FF938091B900887F803609F49CC0D0
:101C200068F5883209F45BC090F4803109F454C03F
:101C300038F4882309F4F5C0883009F44DC0F5C0A4
:101C4000883109F44CC0803209F45DC0EEC08034A4
:101C500009F468C048F4803309F455C0883309F0AA
:101C6000E4C080937003A8C0803509F44FC0883564
:101C700009F45DC0883409F0D8C0D5C0883909F4AA
:101C8000C6C0A8F4883709F467C038F4883609F468
:101C900063C0803709F460C0C8C0883809F4B7C091
:101CA000803909F45FC0803809F0BFC05BC0803B59
:101CB00009F485C038F4803A09F466C0883A09F41A
:101CC0007EC0B3C0803C09F4A6C0883C09F4A3C020
:101CD000883B09F489C0A9C08091DC0310C09091B1
:101CE000B5038091B403981770F5E091B50381E0D6
:101CF0008E0F8093B503F0E0EA54FC4F808180930F
:101D0000BB0085EC85C0809370038DC0E091B50366
:101D100081E08E0F8093B5038091BB00F0E0EA5420
:101D2000FC4F80839091B5038091B4036DC0E09126
:101D3000B50381E08E0F8093B5038091BB00F0E086
:101D4000EA54FC4F80838091DB0381116CC081E0F9
:101D50008093DA0384EA60C083E08093DD0310920D
:101D60007103CFCF80917103803208F050C0E091B1
:101D7000710381E08E0F809371038091BB00F0E0CE
:101D8000EE58FC4F8083BDCF80917103803230F4D8
:101D9000E0917103F0E0EE58FC4F10820E94E90DD3
:101DA0006091710370E0E091D603F091D70382E770
:101DB00093E00995109271030E94F30D36C084E000
:101DC0008093DD031092930310929203E091D80365
:101DD000F091D903099580919203811105C081E0AA
:101DE0008093920310929403E091930381E08E0F0D
:101DF00080939303F0E0EC56FC4F80818093BB000E
:101E00009091930380919203981708F47ACF85E814
:101E10008093BC000AC085EC8093BC001092DD0367
:101E200004C0109270030E94E90DFF91EF91BF91E1
:101E3000AF919F918F917F916F915F914F913F9162
:101E40002F910F900FBE0F901F9018950F931F9317
:101E5000CF93DF93EC018B0188819981DC01ED91B7
:101E6000FC916F770190F081E02D0995888199812F
:101E7000DC01ED91FC91B801660F672F661F770BAF
:101E80006F770190F081E02DDF91CF911F910F913D
:101E90000994DC018D919C91DC01ED91FC91019004
:101EA000F081E02D60EF0994DC018D919C91DC01C3
:101EB000ED91FC910190F081E02D67EF0994CF93B3
:101EC000DF93EC0188819981DC01ED91FC91019017
:101ED000F081E02D69EF099588819981DC01ED9110
:101EE000FC910190F081E02D62E009958881998153
:101EF000DC01ED91FC910190F081E02D64E0DF9137
:101F0000CF9109941F93CF93DF93EC018A818823AB
:101F1000D9F1CE010E94490F88819981DC01ED91B0
:101F2000FC910190F081E02D69E709958881998104
:101F3000DC01ED91FC91AB81BC810190F081E02D41
:101F40006C91099588819981DC01ED91FC91AB81BF
:101F5000BC810190F081E02D11966C91099512E001
:101F60008A81181758F4EB81FC81E10FF11D608123
:101F700070E0CE010E94260F1F5FF2CFCE01DF91ED
:101F8000CF911F910C94540FDF91CF911F91089521
:101F9000CF92DF92EF92FF920F931F93CF93DF9335
:101FA0008C01EB01C42ED22E6BEC71E0CE010E94AD
:101FB000701E7C016FE270E0CE010E94651E0097EA
:101FC00039F46CE570E0CE010E94651E009711F0B7
:101FD000EC012196E114F10451F4FE01019000207E
:101FE000E9F7EC1BEF5FD8011296EC9306C0EC1AF0
:101FF000FD0AE394E394F801E282D80113968D91EF
:102000009C9114970E94C71DF801E280F12CC70132
:1020100001960E942F1DD80114969C938E931397BE
:10202000FC01EE0DFF1D1082FC01C082D1821296D0
:102030004C9150E042505109BE010296DF91CF9180
:102040001F910F91FF90EF90DF90CF900C94561E50
:10205000DC018D919C91DC01ED91FC910480F58176
:10206000E02D09940F931F93CF93DF93FC012085FC
:10207000213749F0293709F049C0DF91CF911F91ED
:102080000F910C94820FFC01E95AFF4F0190F081EF
:10209000E02D309709F450C0DC01A75BBF4F4D9194
:1020A0005C919A012150310937FD9A01B90175956A
:1020B0006795062F40E050E020E030E04E5F5F4F34
:1020C0002017A0F4EC01C40FD51F1F81DC01A20F63
:1020D000B31F18961C931897C885D0E8CD9F101988
:1020E000112418961C932F5F3F4FE8CFDC01A60FF9
:1020F000B11D17962C911797222311F018961C9258
:102100000896DF91CF911F910F910994FC01E75A36
:10211000FF4F0190F081E02D309771F0AC01475FE7
:102120005F4FDC01A75BBF4F6C916150822FDF9145
:10213000CF911F910F910994DF91CF911F910F9132
:1021400008950F931F93CF93DF93EC018A01888149
:102150009981DC01ED91FC916F70606E0190F081CE
:10216000E02D0995B801CE01DF91CF911F910F911C
:102170000C94260F0F931F93CF93DF93EC018A01EA
:1021800088819981DC01ED91FC916F70606901900B
:10219000F081E02D099588819981DC01ED91FC9118
:1021A000602F6F770190F081E02D099588819981EA
:1021B000DC01ED91FC91B801660F672F661F770B6C
:1021C0000190F081E02DDF91CF911F910F91099443
:1021D000CF92DF92EF92FF920F931F93CF93DF93F3
:1021E00000D01F92CDB7DEB78C01F42E2A833B833B
:1021F00069830E94490FD8018D919C91DC01ED917A
:10220000FC910190F081E02D698109952A81E22EEF
:10221000C22E3B81D32E8C2D8E198F1540F4F601E2
:1022200061916F0170E0C8010E94260FF4CFC801D0
:102230000F900F900F90DF91CF911F910F91FF9012
:10224000EF90DF90CF900C94540F9A01FA01019017
:102250000020E9F73197E41BF50B4E2F0C94E810A2
:10226000AB0161E70C942511DC018D919C91DC019F
:10227000ED91FC910190F081E02D0994603DB9F061
:1022800028F4603961F0603C71F00895603E19F007
:10229000643F89F00895FC01E55BFF4F0FC0FC012E
:1022A000E35BFF4F0BC0FC01E15BFF4F07C0FC018C
:1022B000EF5AFF4F03C0FC01ED5AFF4F518340839B
:1022C00008956F3F29F4FC01EB5AFF4F518340837F
:1022D0000895875A9F4FFC01518340830895FC0164
:1022E00015821682178280E090E0DF01A80FB91FE7
:1022F00018961C92019680349105B9F7DF01A85B0E
:10230000BF4F1C9211961D921C92EB5AFF4F0190E9
:10231000F081E02D309709F009940895FC011282B4
:10232000148213820C946F11CF93DF93EC01888198
:102330009981DC01ED91FC910680F781E02D0995F2
:10234000FE01E85BFF4F20812223B1F0873F91051A
:1023500031F41082CE01DF91CF910C943210FE0146
:10236000E75BFF4F20813181C20FD31F88872F5F2A
:102370003F4F318320839DC02D81222309F45EC00D
:10238000803891050CF05AC09FEF920F9D83FE019B
:10239000E90FF11D808791118CC08E81882309F48B
:1023A00088C0803DE9F148F48039E9F0803C09F0CB
:1023B00043C0FE01E15BFF4F36C0803E19F0843F11
:1023C00019F13AC0FE01E55BFF4F0190F081E02D6D
:1023D000309791F18885698570E0B0E88B9F600D3A
:1023E000711D112427C0FE01E35BFF4F0190F081B6
:1023F000E02D309709F18885698570E090E8899F24
:10240000600D711D112416C0FE01ED5AFF4F0190A1
:10241000F081E02D309781F0688570E089850BC0F0
:10242000FE01EF5AFF4F0190F081E02D309721F02F
:10243000688570E08F8109951E823BC0803F9105C1
:102440002CF4282F2F702F83807F9927803E9105B1
:1024500021F154F4803C910511F1803D9105F9F092
:102460008039910531F519C0843F9105B1F054F4DC
:10247000803F9105F1F481E08083C75BDF4F1982D3
:10248000188217C0893F910571F08F3F910589F43B
:10249000CE01DF91CF910C946F1192E001C091E0D9
:1024A0009D838E8306C08EED93E0DF91CF910C94D7
:1024B0005F0FDF91CF9108958F929F92AF92BF925D
:1024C000CF92DF92EF92FF921F93CF93DF93EB01B6
:1024D0004A01690161E08DE00E94021510E0EE24DE
:1024E000D7FCE094FE2CAA2497FCA094BA2C812F50
:1024F00090E08C179D0794F4C701B6010E947613F3
:1025000061E08DE00E943B15C501B4010E94761385
:1025100060E08DE00E943B151F5FE9CFDF91CF9116
:102520001F91FF90EF90DF90CF90BF90AF909F9062
:102530008F900895CF93DF93EC0161E08DE00E94CE
:10254000021522ED30E048E250E062E070E0CE019A
:102550000E945C126AEF70E080E090E00E947613C7
:1025600022ED30E048E250E064E070E0CE010E94ED
:102570005C126DE770E080E090E0DF91CF910C9409
:102580007613CF93DF93EC0188E494E00E94571612
:1025900088E494E099838883CE010E949A12CE0148
:1025A0000E945F0FCE01DF91CF910C94820F8EEDD0
:1025B00093E00C948E110F9300E020E040E060E087
:1025C00089E394E00E94B4160F9108950E94A71326
:1025D0008EE994E00E94071B89B5806189BD09B42A
:1025E00000FEFDCF0E948306C0E0D0E00E94A0095B
:1025F0002097E1F30E940000F9CF1F920F920FB6CF
:102600000F9211242F933F938F939F93AF93BF9378
:102610008091400490914104A0914204B091430400
:1026200030913F0426E0230F2D3720F40296A11DA0
:10263000B11D05C029E8230F0396A11DB11D2093EC
:102640003F048093400490934104A0934204B093CC
:1026500043048091440490914504A0914604B091B4
:1026600047040196A11DB11D809344049093450435
:10267000A0934604B0934704BF91AF919F918F916F
:102680003F912F910F900FBE0F901F9018952FB76D
:10269000F8946091400470914104809142049091BB
:1026A00043042FBF08953FB7F8948091440490915C
:1026B0004504A0914604B091470426B5A89B05C0E7
:1026C0002F3F19F00196A11DB11D3FBF6627782F3E
:1026D000892F9A2F620F711D811D911D43E0660F96
:1026E000771F881F991F4A95D1F70895CF92DF92DF
:1026F000EF92FF92CF93DF936B017C010E94531303
:10270000EB01C114D104E104F10489F00E946E1BB5
:102710000E9453136C1B7D0B683E734090F381E065
:10272000C81AD108E108F108C851DC4FEACFDF919F
:10273000CF91FF90EF90DF90CF9008958330910577
:1027400028F0880F991F04970197F1F7089578945E
:1027500084B5826084BD84B5816084BD85B58260A6
:1027600085BD85B5816085BDEEE6F0E08081816044
:102770008083E1E8F0E01082808182608083808144
:1027800081608083E0E8F0E0808181608083E1E91E
:10279000F0E0808182608083808181608083E0E9D5
:1027A000F0E0808181608083E1ECF0E080818460F2
:1027B0008083808182608083808181608083E3EC7C
:1027C000F0E0808181608083E0ECF0E080818260D5
:1027D0008083E2ECF0E0808181608083EAE7F0E0D2
:1027E00080818460808380818260808380818E7F0D
:1027F00080838081806880830895823108F08251CF
:10280000E82FF0E0E45FFE4FE49180917B00E3FB72
:10281000222720F930E095E0220F331F9A95E1F747
:102820008F7D822B80937B00E77080910D0120E4E7
:10283000829FC0011124E82BE0937C0080917A00F4
:10284000806480937A0080917A0086FDFCCF80912D
:1028500078002091790090E0922B08951F93CF93F8
:10286000DF93182FEB0161E00E940215209711F40D
:1028700060E004C0CF3FD10539F461E0812FDF91E2
:10288000CF911F910C943B15E12FF0E0E85EFE4FD5
:10289000449150E0FA013197EF30F10508F06CC037
:1028A000E859FF4F0C940F1D84B5806884BDC7BDE7
:1028B00068C084B5806284BDC8BD63C0809180005B
:1028C000806880938000D0938900C093880059C0AD
:1028D00080918000806280938000D0938B00C093B1
:1028E0008A004FC080918000886080938000D093E0
:1028F0008D00C0938C0045C08091900080688093CB
:102900009000D0939900C09398003BC080919000B4
:10291000806280939000D0939B00C0939A0031C056
:1029200080919000886080939000D0939D00C09328
:102930009C0027C08091C00080688093C000809177
:10294000C0008F7B8093C000C093CF001AC08091DD
:10295000C00080628093C000C093D00012C08091FC
:10296000C20088608093C2008091C2008B7F8093F8
:10297000C200C093D20005C0C038D1050CF07DCF95
:1029800077CFDF91CF911F91089590E0FC013197AF
:10299000EF30F105B0F5E958FF4F0C940F1D809111
:1029A00080008F7703C0809180008F7D80938000AE
:1029B000089580918000877FF9CF84B58F7702C01A
:1029C00084B58F7D84BD0895809190008F7707C076
:1029D000809190008F7D03C080919000877F8093CD
:1029E000900008958091C0008F7703C08091C0004F
:1029F0008F7D8093C00008958091C200877F80936F
:102A0000C2000895CF93DF9390E0FC01EA5CFE4F93
:102A10002491FC01EC5AFE4F8491882349F190E007
:102A2000880F991FFC01E257FE4FA591B491805881
:102A30009E4FFC01C591D4919FB7611108C0F894D5
:102A40008C91209582238C93888182230AC06230E6
:102A500051F4F8948C91322F309583238C93888194
:102A6000822B888304C0F8948C91822B8C939FBF17
:102A7000DF91CF9108950F931F93CF93DF931F9210
:102A8000CDB7DEB7282F30E0F901E85EFE4F849124
:102A9000F901EA5CFE4F1491F901EC5AFE4F0491E2
:102AA0000023C9F0882321F069830E94C51469813D
:102AB000E02FF0E0EE0FFF1FE058FE4FA591B4911C
:102AC0009FB7F8948C91611103C01095812301C0C8
:102AD000812B8C939FBF0F90DF91CF911F910F910E
:102AE0000895CF93DF93282F30E0F901E85EFE4F81
:102AF0008491F901EA5CFE4FD491F901EC5AFE4F42
:102B0000C491CC2391F081110E94C514EC2FF0E008
:102B1000EE0FFF1FEE58FE4FA591B4912C912D237F
:102B200081E090E021F480E002C080E090E0DF915D
:102B3000CF910895CF93DF931F92CDB7DEB769830E
:102B4000DC01ED91FC910280F381E02D41E050E049
:102B5000BE016F5F7F4F09950F90DF91CF91089570
:102B6000CF93DF93EC018C859D8597FF05C082E0B4
:102B70000E9452189D878C878C859D85DF91CF910F
:102B8000089583E00C94A71AFC018485958597FD30
:102B900006C082E00E94FA1790E00196089582E054
:102BA0000E94FA1790E00895FC018485958597FDB1
:102BB00005C02FEF3FEF35872487089582E00C94FE
:102BC0005218CF93DF93EC0180911501882331F0E7
:102BD00083E00E9483181816190634F081E090E013
:102BE0009B838A8380E090E0DF91CF910895FC0180
:102BF00020812E5F208342E450E06CE971E080E8A0
:102C00000C941E19FC0181819081913A59F4813212
:102C100009F03CC047E050E06EE071E080E00E94C7
:102C20001E1943C0913291F5803239F467E070E0AB
:102C30008EE091E00E944F1906C0823209F035C043
:102C400082818093150180910E0190910F01A091D6
:102C50001001B0911101803B9440A105B105C1F470
:102C60008091150180FD14C087E797E790930108D4
:102C7000809300082BE088E190E00FB6F894A895C7
:102C8000809360000FBE209360000FC080E0089525
:102C900088E10FB6F89480936000109260000FBE38
:102CA000A895109201081092000881E008952FEF76
:102CB0003FEFFC0135872487089510924B04109252
:102CC0004A0488EE93E0A0E0B0E080934C04909337
:102CD0004D04A0934E04B0934F0484ED91E0909383
:102CE0004904809348048FEF9FEF9093550480939D
:102CF00054040895AF92BF92CF92DF92EF92FF9269
:102D00000F931F93CF93DF936C017B01C0E0D0E062
:102D100000E010E0F601EC0FFD1F4AE050E0628198
:102D2000C7010E947A175C016EE2C7010E940D176D
:102D30008A0D9B1D080F191F2196C330D10551F72D
:102D40004AE050E0F6016581C7010E947A17800FC2
:102D5000911FDF91CF911F910F91FF90EF90DF9026
:102D6000CF90BF90AF9008950F93FC0184EE91E057
:102D70009183808362834383248305830F91089525
:102D800084EE91E0909399048093980410929A04B1
:102D900010929B0410929C0410929D040895CF926F
:102DA000DF92EF92FF920F931F93CF93DF936C010B
:102DB0007A01EB01E60EF71E00E010E0CE15DF050C
:102DC00061F06991D601ED91FC910190F081E02DC7
:102DD000C6010995080F191FF1CFC801DF91CF91E6
:102DE0001F910F91FF90EF90DF90CF9008956115A4
:102DF000710581F0DB010D900020E9F7AD01415034
:102E00005109461B570BDC01ED91FC910280F381C7
:102E1000E02D099480E090E00895DC01ED91FC91B3
:102E20000190F081E02D09948F929F92AF92BF9212
:102E3000CF92DF92EF92FF920F931F93CF93DF9386
:102E4000CDB7DEB7A1970FB6F894DEBF0FBECDBFEA
:102E50007C01C42EE52FCB01D22E19A221E02D1525
:102E600010F02AE0D22E8E010F5D1F4F8D2C912C79
:102E7000A12CB12C6C2D7E2FA50194010E94CE1C9B
:102E80008C2DD29E80191124015011098A3014F41E
:102E9000805D01C0895CF801808321153105410501
:102EA000510521F0C22EE32FCA01E4CFB801C701BA
:102EB0000E94F716A1960FB6F894DEBF0FBECDBFE5
:102EC000DF91CF911F910F91FF90EF90DF90CF9006
:102ED000BF90AF909F908F9008952115310541F4D8
:102EE000DC01ED91FC910190F081E02D642F0994BB
:102EF0000C9414179A01462F50E060E070E00C9497
:102F00006D174091A2045091A3042091A004309128
:102F1000A10442175307B4F49091E8009570E1F3CF
:102F20009091E80092FD19C08093F1008091A20475
:102F30009091A30401968F739927892B19F48EEF32
:102F40008093E8008091A2049091A304019690934D
:102F5000A3048093A20481E0089580E00895CF92B5
:102F6000DF92FF920F931F93CF93DF931F92CDB702
:102F7000DEB7082F162F862F880F8E5F99830E9449
:102F8000811783E00E948117F02EC02E9981D92EDF
:102F90008C2D8F19811778F4F60184910E94811786
:102FA000082F80E00E9481178023FFEFCF1ADF0AED
:102FB0008111EECF01C081E00F90DF91CF911F9181
:102FC0000F91FF90DF90CF900895615030F02091E5
:102FD000F100FC0120830196F8CF289A84E68093C3
:102FE000A50408952FB7FC012083F89467706093BF
:102FF000E9000895CF93DF931F92CDB7DEB7682F16
:10300000CE0101960E94F2178091F20099819FBF34
:103010000F90DF91CF910895FF920F931F93CF935D
:10302000DF9300D0CDB7DEB7F62E8A019091A404CD
:10303000992311F057FF03C08FEF9FEF2BC0682F2C
:10304000CE0101967A830E94F2178091F20090E0FF
:10305000A8017A81801791070CF4AC01EF2DF72FAE
:10306000F40E84E6FE1639F0289A8093A504909118
:10307000F1009193F7CF4115510521F08091F200B5
:10308000882321F089818FBFCA0104C08BE6809319
:10309000E800F8CF0F900F90DF91CF911F910F9123
:1030A000FF900895CF93DF931F92CDB7DEB741E035
:1030B00050E0BE016F5F7F4F0E940C18019719F41A
:1030C000898190E002C08FEF9FEF0F90DF91CF9149
:1030D0000895CF93DF931F92CDB7DEB7682FCE014F
:1030E00001960E94F2179091E800892F807295FF57
:1030F00004C09091F20080E4891B99819FBF0F90DA
:10310000DF91CF9108956F927F928F929F92AF92AD
:10311000BF92CF92DF92EF92FF920F931F93CF93C4
:10312000DF931F92CDB7DEB7782E7B01C42EB52E6C
:103130008091A404882369F0042F152F8AEFD82EDC
:10314000872D8072982E9AE3A92E872D8074882E61
:1031500011C08FEF9FEF57C0872D0E946918682E0E
:1031600081110CC0DA94A9F361E070E080E090E096
:103170000E9476130115110579F73BC0282F30E026
:10318000021713070CF4602E672DCE0101960E94E2
:10319000F2178091E80085FF29C0262D30E0021B40
:1031A000130B992039F06A948FEF6816B1F01092E2
:1031B000F100F9CFF701862D77FE07C0815058F056
:1031C00094919093F1003196F9CF815020F0919134
:1031D0009093F100FACFE20EF31E8091E80085FF94
:1031E0000FC00115110511F481100AC089818FBF2C
:1031F000C1CF5D9A84E68093A6048C2D9B2D03C0DD
:10320000A092E800F3CF0F90DF91CF911F910F9123
:10321000FF90EF90DF90CF90BF90AF909F908F90F6
:103220007F906F9008951092E9001092A30410927D
:10323000A2049093A1048093A0040895CF92DF92FA
:10324000FF920F931F93CF93DF9300D0CDB7DEB7DC
:10325000F82E8A016B0101151105B1F0F601F7FE98
:1032600002C0849101C0808149835A830E948117E2
:1032700001501109FFEFCF1ADF0A49815A818111EC
:10328000EACF8FEF9FEF01C0CA010F900F90DF913F
:10329000CF911F910F91FF90DF90CF9008951F93D2
:1032A000CF93DF931F92CDB7DEB7162F2091E800A2
:1032B00022FFFCCF612F79830E94E5178BEF80936B
:1032C000E800812F7981972F0F90DF91CF911F9187
:1032D0000895CF93DF931F92CDB7DEB71982CE0149
:1032E00001960E94F715CE0101960E948D1B8981DF
:1032F00090E00F90DF91CF9108951F920F920FB63B
:103300000F921124EF92FF920F931F932F933F93ED
:103310004F935F936F937F938F939F93AF93BF93DD
:10332000EF93FF93CF93DF93CDB7DEB76297DEBF06
:10333000CDBF1092E9008091E80083FFEBC068E008
:10334000CE010A960E94E51782EF8093E8009A85E5
:1033500097FF05C08091E80080FFFCCF03C08EEF8F
:103360008093E800892F807609F0B9C08B858111A0
:1033700005C01092F1001092F100C5C0282F2D7FDA
:10338000213009F4C0C0853049F48091E80080FF05
:10339000FCCF8C8580688093E300B5C0863009F04F
:1033A00076C02D85E888F988223071F580E090E0BC
:1033B0002A8B0E9413190E94691999E08E010F5FF0
:1033C0001F4FF801392F11923A95E9F799832A890D
:1033D0002A8391E09E8390E898879AEF99872091BD
:1033E000A2043091A304275F3F4F3C832B838D833E
:1033F000C7010E94131949E050E0B80180E00E9423
:103400001E190E9469197FC0C7012A8B0E941319D7
:103410002A89223241F482E290E00E94981B892B93
:1034200009F071C074C0213069F4888999890897BE
:1034300011F420939F0480919F04811118C065EFBF
:1034400071E01AC0233009F062C08C85882391F0A6
:10345000823021F46BE08BE092E006C0813009F00D
:1034600056C063E087E092E00E94AF174AC063EE67
:1034700071E002C067E172E06115710509F447C0AF
:10348000FB01449150E080E80E941E193CC0873047
:1034900009F43DC0883021F481E08093F10033C00D
:1034A000893089F5937099F5EFEDF1E081E021E045
:1034B00096E38093E9002093EB0034913093EC0085
:1034C0009093ED008F5F3196853099F78EE780936A
:1034D000EA001092EA008C858093A40414C08889C5
:1034E00099890E9413198E85811105C0CE010A9613
:1034F0000E94021606C0823051F4CE010A960E9444
:10350000C01B882321F08EEF8093E80003C081E286
:103510008093EB0062960FB6F894DEBF0FBECDBF6E
:10352000DF91CF91FF91EF91BF91AF919F918F91DB
:103530007F916F915F914F913F912F911F910F91CB
:10354000FF90EF900F900FBE0F901F9018958093F3
:10355000E9008091F200882319F08AE38093E80063
:1035600008951F920F920FB60F9211242F933F933D
:103570004F935F936F937F938F939F93AF93BF937B
:10358000EF93FF938091E1001092E10083FF0FC061
:103590001092E90091E09093EB001092EC0092E31E
:1035A0009093ED001092A40498E09093F00082FFB5
:1035B0001DC083E00E94A71A8091A604882339F0D9
:1035C0008091A60481508093A604882369F080919D
:1035D000A504882359F08091A50481508093A50407
:1035E000811104C0289802C05D98F1CFFF91EF913E
:1035F000BF91AF919F918F917F916F915F914F910B
:103600003F912F910F900FBE0F901F901895109221
:10361000A40481E08093D70080EA8093D80082E000
:1036200089BD09B400FEFDCF61E070E080E090E06C
:103630000E94761380E98093D8008CE08093E200AA
:103640001092E000559A209A5D98289808954F921C
:103650005F926F927F92AF92BF92CF92DF92EF9282
:10366000FF920F931F93CF93DF93CDB7DEB729015E
:103670003A01621B730B840B950B29893A894B899C
:103680005C892A193B094C095D09298B3A8B4B8BC4
:103690005C8B9B01AC0169897A898B899C890E942A
:1036A000B21CE418F50806091709A80197010E9441
:1036B000F01C2A0D3B1D4C1D5D1DCA01B901DF9197
:1036C000CF911F910F91FF90EF90DF90CF90BF901F
:1036D000AF907F906F905F904F9008950895FF9204
:1036E0000F931F93CF93DF93EC01F62EE881F981BE
:1036F0000480F581E02D09958C01E881F98106802F
:10370000F781E02D6F2DCE010995C8019927DF9132
:10371000CF911F910F91FF900895FC0120812F5FA1
:10372000208349E150E06BE972E080E80C941E19B7
:1037300045E650E064EB72E080E80C941E19EF92CD
:10374000FF920F931F93CF93DF931F92CDB7DEB7F6
:1037500089838B017A0141E050E0BE016F5F7F4FAA
:1037600084E00E948318A701B80184E40E948318B2
:103770000F90DF91CF911F910F91FF90EF900895DF
:10378000FC0191818081813A31F481E0913091F0A6
:10379000933089F411C0813271F49B3021F482811D
:1037A0008093170105C09A3031F48281809316010D
:1037B00081E00895089580E0089548E050E082E0B7
:1037C0000C949F1BCF93DF93DC01683818F0E8E777
:1037D000E60F25C0E62FF0E067FF11C0E058F109C1
:1037E00081E090E001C0880FEA95EAF714969C9179
:1037F0001497982B14969C931497E0E010C0E55E04
:10380000FD4FE491EE2309F440C0E7FF08C0149691
:103810008C911497826014968C931497EF77169678
:103820008C9116978E1741F117968C9117978E17DA
:1038300019F118968C9118978E17F1F019968C91B2
:1038400019978E17C9F01A968C911A978E17A1F0B6
:103850001B968C911B978E1779F080E090E0ED011C
:10386000C80FD91F2E81211102C0EE8305C0019619
:1038700086309105A1F709C0BD016C5F7F4FCD0176
:103880000E94DD1B81E090E008C081E090E013968B
:103890009C938E93129780E090E0DF91CF910895F2
:1038A000683818F0E8E7E60F25C0E62FF0E067FF7C
:1038B00012C0E058F10921E030E001C0220FEA9582
:1038C000EAF72095DC0114963C9114973223149664
:1038D0003C93E0E00FC0E55EFD4FE491EE2329F15B
:1038E000E7FF08C0DC0114962C9114972D7F1496E5
:1038F0002C93EF7720E030E0EE2351F0DC01A20FB3
:10390000B31F16964C9116974E1302C016961C9232
:103910002F5F3F4F2630310579F7BC016C5F7F4F39
:103920000E94DD1B81E090E0089580E090E0089522
:10393000FC01168217821086118612861386148265
:10394000BC016C5F7F4F0C94DD1B1092B30410928E
:10395000AA041092A9048AEE91E09093A80480939F
:10396000A7040895DB018F939F930E94151DBF91BB
:10397000AF91A29F800D911DA39F900DB29F900DBE
:1039800011240895991B79E004C0991F961708F037
:10399000961B881F7A95C9F780950895A1E21A2E83
:1039A000AA1BBB1BFD010DC0AA1FBB1FEE1FFF1FE3
:1039B000A217B307E407F50720F0A21BB30BE40B33
:1039C000F50B661F771F881F991F1A9469F760957A
:1039D0007095809590959B01AC01BD01CF01089534
:1039E000052E97FB1EF400940E94071D57FD07D07B
:1039F0000E94CE1C07FC03D04EF40C94071D50957A
:103A00004095309521953F4F4F4F5F4F08959095CA
:103A10008095709561957F4F8F4F9F4F0895EE0F62
:103A2000FF1F0590F491E02D09940E94201DA59F91
:103A3000900DB49F900DA49F800D911D11240895A9
:103A4000A29FB001B39FC001A39F700D811D1124DF
:103A5000911DB29F700D811D1124911D0895CF936A
:103A6000DF938230910510F482E090E0E091B6049B
:103A7000F091B70420E030E0A0E0B0E0309739F1F9
:103A80004081518148175907B8F04817590771F418
:103A900082819381109729F013969C938E931297AD
:103AA0002CC09093B7048093B60427C0211531052C
:103AB00031F04217530718F0A901DB0101C0EF01F3
:103AC0009A01BD01DF010280F381E02DD7CF2115DE
:103AD0003105F9F0281B390B2430310580F48A8137
:103AE0009B816115710521F0FB019383828304C0E2
:103AF0009093B7048093B604FE01329644C0FE0151
:103B0000E20FF31F81939193225031093983288367
:103B10003AC02091B4043091B504232B41F4209194
:103B20000201309103013093B5042093B404209135
:103B30000001309101012115310541F42DB73EB747
:103B40004091040150910501241B350BE091B40410
:103B5000F091B504E217F307A0F42E1B3F0B2817D2
:103B6000390778F0AC014E5F5F4F2417350748F0F6
:103B70004E0F5F1F5093B5044093B404819391930B
:103B800002C0E0E0F0E0CF01DF91CF910895CF9344
:103B9000DF93009709F487C0FC01329713821282E9
:103BA000C091B604D091B704209781F4208131816F
:103BB000280F391F8091B4049091B50482179307A0
:103BC00079F5F093B504E093B4046DC0DE0120E014
:103BD00030E0AE17BF0750F412964D915C911397E9
:103BE0009D014115510509F1DA01F3CFB383A28399
:103BF00040815181840F951F8A179B0771F48D9125
:103C00009C911197840F951F029691838083129641
:103C10008D919C911397938382832115310529F40B
:103C2000F093B704E093B6043EC0D9011396FC9319
:103C3000EE9312974D915D91A40FB51FEA17FB0704
:103C400079F480819181840F951F0296D901119694
:103C50009C938E938281938113969C938E9312975B
:103C6000E0E0F0E08A819B81009719F0FE01EC0111
:103C7000F9CFCE01029628813981820F931F2091BE
:103C8000B4043091B5042817390769F4309729F442
:103C90001092B7041092B60402C013821282D0931D
:103CA000B504C093B404DF91CF910895FB01DC010A
:103CB0004150504048F001900D920020C9F701C0DA
:103CC0001D9241505040E0F70895FC0181E090E0E2
:103CD0000190061609F4CF010020D1F7019708954D
:103CE000FB0151915523A9F0BF01DC014D9145170E
:103CF0004111E1F759F4CD010190002049F04D91B7
:103D000040154111C9F3FB014111EFCF81E090E073
:083D100001970895F894FFCF1C
:103D18000000B804800001000000FF13000100E16A
:103D280000000000000001014D6178207365727683
:103D38006F7320617474616368656400556E6B6E9F
:103D48006F776E2070696E206D6F646500537461C3
:103D58006E646172644669726D6174612E696E6F1A
:103D6800004932433A20546F6F206D616E792062AA
:103D78007974657320726563656976656400493294
:103D8800433A20546F6F20666577206279746573B3
:103D98002072656365697665640031302D626974E7
:103DA8002061646472657373696E67206E6F742036
:103DB800737570706F7274656400746F6F206D61D5
:103DC8006E79207175657269657300000000009E48
:103DD8000C710C460C4E0C610C700C2E637070004C
:103DE800000000009A15E115C415D415B015C115C9
:103DF800000000007A16000000006F1BCF16E21BBF
:043E0800501C981C96
:00000001FF
